:100000000C9419030C9436030C9436030C94031EC1
:100010000C9436030C9436030C9436030C9436037C
:100020000C9436030C9436030C941F260C94F12682
:100030000C944C200C9436030C9436030C94360329
:100040000C9436030C9436030C9436030C9436034C
:100050000C9436030C94F0200C9436030C94360365
:100060000C9436030C9436030C9436030C9436032C
:100070000C9436030C9436030C9436030C9436031C
:100080000C9436030C9436030C9436030C9436030C
:100090000C9436030C9436030C9436030C943603FC
:1000A0000C9436030C9436030C94360377067706CB
:1000B000A306A3060B072907410841083407CD070B
:1000C000DE07DE075E2785277D2885277D28D12747
:1000D000F4277D284B285A282200210020001F00E9
:1000E0001E00290000000000000017001500080095
:1000F0001A0014002B000000000000000A00090094
:10010000070016000400E0000000000000000500E9
:10011000190006001B001D00E100000000000000A7
:100120002C00E300E200E0000000000000000000FE
:1001300000002F0000000000000000000000000090
:1001400000000000230024002500260027002A00CC
:100150002D002E0035001C0018000C0012001300AA
:100160004C002F00300031000B000D000E000F007E
:10017000330034000000520000001100100036006F
:1001800037003800E500500051004F0028000251B0
:1001900001510000000000000000000000003000DD
:1001A000000000000000000000000000000000004F
:1001B00001000100010001000100005C00000000DE
:1001C0000000010001000100010001000100000029
:1001D0000000000001000100010001000100010019
:1001E000000000000000010001000100010001000A
:1001F00001000000000000000100010001000100FA
:1002000000000000000000000000010000000000ED
:1002100000000000000000000000000001000100DC
:100220000100010001000100A800AA00A9000100CE
:1002300001000100010001000100010001000100B6
:1002400001000100010001000100010000000100A7
:100250000000010001000100010001000100010097
:100260000100010001000100010001000000000088
:10027000000000000000010000000000000000007D
:10028000000000000000000001000100010001006A
:100290000100010000000000000001000100010059
:1002A0000100010001000000000000000100010049
:1002B0000100010001000100000000000000010039
:1002C0000100010001000100010000000000000029
:1002D000010001000100010000000000000000001A
:1002E000000001000000000000000000000000000D
:1002F0000000000001006700540055005600010096
:1003000001000100010001005F0060006100570072
:10031000010001000100010001005C005D005E00C1
:1003200001000100000001000000010059005A0016
:100330005B0001000100010001000100010001005B
:1003400062006300000000000000000000000100E7
:10035000000000000000000000000000000000009D
:1003600044454255473A2064697361626C65642E66
:100370000A0044454255473A20656E61626C6564E7
:100380002E0A000A0025303258006C65645F7461E3
:10039000736B3A20004F6E6573686F743A20616327
:1003A000746976653A2025640A000A0025303136E2
:1003B00062003A200025303258000A722F63203044
:1003C0003132333435363738394142434445460AB1
:1003D0000054617267657420636F6E6E6563746547
:1003E000640D0A0054617267657420646973636FF9
:1003F0006E6E65637465642C207468726F74746CBF
:10040000696E6720636F6E6E656374696F6E2061DD
:100410007474656D7074730D0A004661696C65646F
:1004200020746F20657865637574652025730A00F4
:10043000290A002575002F002575005D2800256418
:1004400000200025640020002564002000256400B1
:100450007C0025303258006D6F7573656B657920AF
:100460005B62746E7C782079207620685D287265E6
:10047000702F61636C293A205B000A0025303258E6
:1004800020006B6579626F6172645F7265706F7274
:10049000743A20005B735D005B575D005B535D0049
:1004A0005B525D005B445D005B435D0018034F00E1
:1004B0006300650061006E00420072006500650027
:1004C0007A00650000001C034100660074006500AE
:1004D00072006E006F006F006E004C0061006200E1
:1004E000730000000403090409025B00030100A07B
:1004F000FA090400000103010100092111010001B2
:1005000022400007058103080001090401000103DE
:10051000000000092111010001227B000705820370
:10052000200001090402000203000000092111015A
:1005300000012222000705830320000107050303B1
:1005400020000112010002000000086C610300019C
:1005500000010200010631FF0974A10109751500AF
:1005600026FF009520750881020976150026FF00F8
:10057000952075089102C005010902A101850209B3
:1005800001A1000509190129081500250195087523
:100590000181020501093009311581257F95027518
:1005A00008810609381581257F95017508810605A2
:1005B0000C0A38021581257F950175088106C0C097
:1005C00005010980A101850319012AB7001501263B
:1005D000B700950175108100C0050C0901A10185C6
:1005E0000419012AA002150126A0029501751081A7
:1005F00000C005010906A101050719E029E715005A
:10060000250195087501810295017508810105078D
:10061000190029FF150026FF0095067508810005C1
:100620000819012905950575019102950175039138
:1006300001C011241FBECFEFDAE0DEBFCDBF11E055
:10064000A0E0B1E0ECEAF2E502C005900D92AC3C0E
:10065000B107D9F723E0ACECB1E001C01D92AF3295
:10066000B207E1F70E94F2170C9454290C94000091
:10067000FF93EF93E091CC01F091CD01309709F019
:100680000995EF91FF910895FC018591803011F05B
:10069000EFDFFBCF0895FF27E0E230E247FF0CC019
:1006A000419597FF09C0EDE2609570958095909512
:1006B000611D711D811D911D27FF02C0219530E331
:1006C00050E2AA27660F771F881F991FAA1FA41739
:1006D00010F0A41B63955A95A9F7AA3008F0A95FFA
:1006E000A05DAF93F395611571058105910541F703
:1006F000ED3211F4EF93F395F21718F43F93F3955D
:10070000FBCF8F91B5DFFA95E1F70895E991F99163
:100710008591803021F0853219F0AADFF9CF089554
:1007200020E0E89455915532C1F3503311F46894A8
:1007300055915A3348F4505390F3220F022E220F52
:10074000220F200D250FF4CF0EF421958991999158
:10075000533619F3533729F1533559F1BC01882722
:100760009927E8945C3621F4899199916894559180
:10077000543639F446EF7EF077FF0DC08FEF9FEFD0
:100780000AC055374AE039F0583540E121F0523679
:1007900042E009F00895FF93EF937DDFEF91FF9121
:1007A000B7CFFF93EF93FC0181918030B9F360DF05
:1007B000FBCFFF93EF9368DFF1CFDF93CF93CDB7FC
:1007C000DEB72596A3DFCF91DF91089581E00895EC
:1007D00081E008950C94E80308950C94EC031F93B2
:1007E000CF93DF9300D000D01F92CDB7DEB74983FF
:1007F0005A836B833091CF0189819A81311114C062
:10080000662359F0222349F00E947E0A182F682F90
:1008100089819A810E94270A03C00E94520A182FD8
:1008200069817A81812F04C00E947E0A69817A8160
:100830000F900F900F900F900F90DF91CF911F911D
:100840000C94D011FC01262F40815181628173816B
:1008500084810C94EF0381E00895CF93DF93EC0142
:1008600060E00E942204BE01DF91CF910C94ED0361
:100870000C94AE130C94AA1308950E94D1080E9400
:100880003C042FEF84E39CE0215080409040E1F74E
:1008900000C000000C9416210F931F93CF93DF9399
:1008A0008C0161E00E942204EC01B8010E94EA037D
:1008B000882309F45BC0B801CE010E940E1D882375
:1008C00009F454C0B801CE010E94221B882309F408
:1008D0004DC0B801CE010E946A1C882309F446C0AD
:1008E000F80182818823D9F1CF3D8CE5D80779F1D1
:1008F00040F4C115FCE5DF0791F0C130DC4591F013
:100900002EC0CC35EDE5DE0741F1CD35FDE5DF0745
:1009100009F1CB35DD4519F50E94150F20C00E9465
:100920003D0424C080918A02C82FC095C170C0FBCD
:1009300080F980938A02CC2329F082E793E00E9419
:10094000440314C080E693E00E94440310C00E9458
:10095000C90F0CC00E940C0F02C00E94180FC801E2
:10096000DF91CF911F910F910C94E603C0E08C2F83
:10097000DF91CF911F910F9108950E942E200C942A
:10098000FB040E94FE040C9434208295982F9373EC
:1009900044E0949F900111248C7C86958695282BA9
:1009A000822F8575880F2A7A2695822B0895CF93FA
:1009B000DF93D92F0E94C504C82F8D2F0E94C50434
:1009C0002C2F30E0322F2227A901482BCA01DF91BA
:1009D000CF91089508950C94EA0481E008950C9451
:1009E000ED040895CF93C82F0E94EB048C2F0E9432
:1009F000EF04CF91089580E00C94F2040E942E1F22
:100A00000C94F204CF930E942E1FC82F8091CE0128
:100A1000C81741F1C093CE0180918A0282FF1EC0A7
:100A200080FF04C08AE893E00E94440380918A0218
:100A300080FF0CC01F92CF9385E893E09F938F9324
:100A40000E94DD030F900F900F900F9080918A020B
:100A500080FF04C083E893E00E9444038C2FCF9171
:100A60000C94F204CF910895CF93DF93CDB7DEB706
:100A70002B970FB6F894DEBF0FBECDBF4F835887BC
:100A800069877A878B8761110E94440E9E012F5FD0
:100A90003F4F86E0F90111928A95E9F785E0FE0162
:100AA0003796D90101900D928A95E1F789819A8153
:100AB0004C815D81452B31F09F3F31F491E08F3FB8
:100AC00019F403C091E001C090E090FF09C0498192
:100AD0005A816B817C818D819E810E94650D05C04C
:100AE000C9010E942B048111F2CF2B960FB6F89406
:100AF000DEBF0FBECDBFDF91CF910895FC01808195
:100B000091810E94C00A0895CF93882309F450C0B0
:100B1000C82F8CEF8C0F813AD0F46C2F809102019A
:100B2000909103010E94D01F882349F06C2F80917F
:100B30000201909103010E9408200E94660E6C2F12
:100B400080910201909103010E9406200CC080E276
:100B50008C0F883058F4C77081E001C0880FCA95A7
:100B6000EAF70E94270ECF910C94660EEBE5EC0F8E
:100B7000E33040F4F0E0E05AFE4F808190E0CF9106
:100B80000C94981FE8E5EC0FE73150F4F0E0EE0F1D
:100B9000FF1FEE5CFE4F80819181CF910C94AE1FC0
:100BA000CD3E30F08C2F0E947718CF910C944919CC
:100BB000CF910895882389F19CEF980F913A40F4E2
:100BC000682F80910201909103010E9408200DC0BE
:100BD00090E2980F983058F4877091E001C0990F17
:100BE0008A95EAF7892F0E942D0E0C94660E9BE5DC
:100BF000980F933020F480E090E00C94981F98E5D3
:100C0000980F973120F480E090E00C94AE1F8D3E59
:100C100020F00E94D2180C94491908951F93CF9385
:100C2000DF93182FEB010E948405209741F08FE994
:100C30009FE00197F1F700C000002197F6CF812FC8
:100C4000DF91CF911F910C94DA05893319F060E0A0
:100C500070E002C060E570E00C940E06882321F07D
:100C60000E94270E0C94660E0895882321F00E949E
:100C70002D0E0C94660E0895CF92DF92EF92FF92A4
:100C80000F931F93CF93DF937C01D62FC72FFC01C7
:100C90001281058102950F700E941D0E8823B9F004
:100CA0001123A9F08C2F807F803421F080E28D0FFA
:100CB000883068F08091EB0282FD09C082E00E94DA
:100CC000C60E0E941D0E91E0D82ED92601C0D12C4F
:100CD000CC2EC2948FE0C8228C2D90E08C309105F0
:100CE00008F0CFC1FC01EA5AFF4F0C94E2288C2F88
:100CF000807FCF70882311F0C295C07F112399F0B7
:100D0000CC2309F4AAC180E28D0F883010F0D111F4
:100D100004C08C2F0E94270E03C08C2F0E94370E18
:100D20000E94660E9AC18D2F0E94DA05CC2309F429
:100D3000A8C180E28D0F883038F1DD2329F18C2F96
:100D40000E943D0E24C08C2F807FCF70803211F026
:100D5000C295C07FDD2319F0D130A1F13DC0809153
:100D6000EB0282FF17C0112349F0CC2329F08C2F0E
:100D70000E94270E0E94660E80E070C180E00E94F3
:100D8000DA05CC2309F47DC18C2F0E942D0E0E9420
:100D9000660E77C1112371F0002341F0013031F468
:100DA0000E94470E8C2B0E944F0E6BC10E94470E73
:100DB0008C2B1DC0002319F0013009F462C10E9480
:100DC0005C0E25C0112321F0063008F05AC10EC078
:100DD000053008F056C11BC0112361F0002331F02B
:100DE000F701858180FF39C18F7085838C2F0E9428
:100DF0002E0647C1002359F0D93309F03FC1FFEF58
:100E000007EE13E0F15000401040E1F735C18C2FA0
:100E10000E94350636C18C2F86958695837019F011
:100E2000813061F02EC1112321F08D2F9C2F937002
:100E300002C080E090E00E94981F2BC1112321F096
:100E40008D2F9C2F937002C080E090E00E94AE1F17
:100E500020C18D2F112319F00E94771802C00E9423
:100E6000D2180E94491915C18C2F837009F047C010
:100E700011110BC12D2F229526952770220F220FBD
:100E80006D2F6F70862F90E0A0E0B0E0022E04C0BE
:100E9000880F991FAA1FBB1F0A94D2F7D4FF10C056
:100EA0004FE050E060E070E004C0440F551F661F43
:100EB000771F2A95D2F7409550956095709503C09D
:100EC00040E050E0BA01C695C695C3708A019B0107
:100ED000082B192B2A2B3B2BC901B801C23049F032
:100EE00058F4C13019F00E943D09CFC00E942B096F
:100EF000CCC00E944F09C9C00E942909C6C0112355
:100F000019F08C2F817001C08695882309F4BDC02B
:100F10002D2F229526952770220F220F6D2F6F708F
:100F2000862F90E0A0E0B0E0022E04C0880F991F49
:100F3000AA1FBB1F0A94D2F7D4FF10C04FE050E0A5
:100F400060E070E004C0440F551F661F771F2A95AC
:100F5000D2F7409550956095709503C040E050E001
:100F6000BA01C695C695C3708A019B01082B192B3F
:100F70002A2B3B2BC901B801C23049F058F4C130CB
:100F800019F00E94020A81C00E94F0097EC00E94EE
:100F9000140A7BC00E94630978C0CF70112339F016
:100FA0008C2F0E9489098D2F0E942E066EC08D2FD6
:100FB0000E9435068C2F0E94AA0967C0D23F21F1FA
:100FC00028F4D03F41F0D13FC1F043C0D33F19F1E5
:100FD000D43F79F03EC0112341F0053008F051C0F4
:100FE0008C2F8F710E94CF094CC0063008F049C089
:100FF000F7CF8091EB0282FF18C0112339F08C2FBC
:101000008F710E9489093DC01123C9F38C2F8F7104
:101010000E94AA0936C0112329F08C2F8F710E94DB
:1010200074092FC00E946F092CC0112349F0CF71A1
:101030008C2F0E94890963E08C2F0E94AB0E21C087
:1010400081E00E94C60E0230E0F082E00E94C60EEF
:1010500018C0112331F0002391F28D2F0E948405D6
:1010600010C0002399F2D93349F41FEF27EE33E083
:10107000115020403040E1F700C000008D2F0E9449
:10108000DA0588EF8C0D843020F40E942E1F0E9418
:10109000F204DD20C9F00E94190E80FD15C0F70191
:1010A00012820E94130E0E948909C7010E948508BE
:1010B0000E94130EDF91CF911F910F91FF90EF903F
:1010C000DF90CF900C94AA09DF91CF911F910F91DF
:1010D000FF90EF90DF90CF9008950F931F93CF93E1
:1010E000DF93EC01688179818A810E94CB0A8C01AF
:1010F0000E94260A0E941709B801CE010E943C06F0
:10110000DF91CF911F910F910895CF93DF93EC0161
:10111000988189812B813C81232B31F08F3F31F4E1
:1011200081E09F3F19F403C081E001C080E080FDB1
:101130001DC0CE010E944C04811110C00E941D0EE2
:101140008823A1F08A81882389F08091EB0282FDB7
:101150000DC082E0DF91CF910C94C60ECE010E94AB
:101160006D08CE01DF91CF910C942D04DF91CF91CA
:10117000089580E090E00E94981F80E090E00E9437
:10118000AE1F0E94440E0E94660E0E94FC1A0C9430
:10119000491980910201909103010E940A200C9448
:1011A000B9080E94340E0C94C90892959F7096302D
:1011B00079F010F4925001C09A50923068F4803F58
:1011C00069F018F4883E40F409C0843F29F406C051
:1011D000883E20F0813F11F080E0089581E008957D
:1011E000FC01808191810E94C00A0E94D508089567
:1011F000CF93DF9300D000D01F92CDB7DEB70F9012
:101200000F900F900F900F90DF91CF910895CF9393
:10121000DF9300D000D000D0CDB7DEB726960FB652
:10122000F894DEBF0FBECDBFDF91CF910895089532
:1012300008950C9418090C9419090E941B096093D5
:101240001A0270931B0280931C0290931D020C944F
:10125000B9080C941D090F931F9300911A02109165
:101260001B0220911C0230911D02602B712B822BDE
:10127000932B1F910F910C941D090F931F930091B5
:101280001A0210911B0220911C0230911D02602352
:101290007123822393231F910F910C941D090F93A7
:1012A0001F9300911A0210911B0220911C02309191
:1012B0001D0260277127822793271F910F910C949D
:1012C0001D090C9418090E9461096093160270931D
:1012D000170280931802909319020C94B90860E0E9
:1012E00070E0CB010C9463090F931F9341E050E031
:1012F00060E070E08A019B0104C0000F111F221FF3
:10130000331F8A95D2F7C901B8011F910F910C9430
:1013100063090F931F9341E050E060E070E004C068
:10132000440F551F661F771F8A95D2F780911602CA
:1013300090911702A0911802B09119028A019B01A5
:10134000082B192B2A2B3B2BC901B8011F910F9198
:101350000C9463090F931F9341E050E060E070E04C
:1013600004C0440F551F661F771F8A95D2F740951A
:101370005095609570958091160290911702A091FA
:101380001802B09119028A019B01082319232A230C
:101390003B23C901B8011F910F910C9463090F936E
:1013A0001F9341E050E060E070E004C0440F551F1F
:1013B000661F771F8A95D2F78091160290911702C7
:1013C000A0911802B09119028A019B0108271927E0
:1013D0002A273B27C901B8011F910F910C9463097B
:1013E0000F931F930091160210911702209118027B
:1013F00030911902602B712B822B932B1F910F912F
:101400000C9463090F931F93009116021091170219
:1014100020911802309119026023712382239323B3
:101420001F910F910C9463090F931F930091160263
:10143000109117022091180230911902602771272C
:10144000822793271F910F910C946309089529E037
:10145000929F800D1124E82FE695E695E69587701A
:1014600051E001C0550F8A95EAF785E0E89FF00149
:101470001124E053FE4F20E030E070E04081CB01CA
:10148000022E02C0969587950A94E2F781708195A5
:1014900084278523842781932F5F3F4F2530310593
:1014A00069F7089529E0929F800D1124682F6695B1
:1014B00066956695982F977085E0689FB001112416
:1014C00040E050E080E0FB01E40FF51FE053FE4FE9
:1014D000208130E0092E02C0369527950A94E2F764
:1014E00021703327042E01C0220F0A94EAF7822BC1
:1014F0004F5F5F4F4530510531F70895BF92CF924E
:10150000DF92EF92FF920F931F93CF93DF938C01A3
:10151000C0901602D0901702E0901802F0901902C5
:1015200080911A0290911B02A0911C02B0911D02A1
:10153000C82AD92AEA2AFB2ACFE1D0E0D701C6017E
:101540000C2E04C0B695A795979587950A94D2F767
:1015500080FD04C0219790F7B12C07C0BC2EB801C4
:101560008C2F0E94E3110197A9F38B2DDF91CF916E
:101570001F910F91FF90EF90DF90CF90BF90089553
:10158000CF93DF93EC010E947E0ABE010E94E3111B
:10159000DF91CF9108951F93CF93DF93EB0190914B
:1015A000CF01992321F0CB010E94C00A13C08823E8
:1015B00049F0CB010E947E0A182F682FCE010E94AD
:1015C000270A04C0CB010E94520A182FBE01812FA6
:1015D0000E94E311DF91CF911F9108951F93CF9344
:1015E000DF93C0911E0216E080911F02C81799F088
:1015F000D0E01C9FF0011D9FF00D1124E05EFD4F17
:101600004081518162817381848195810E940709A3
:101610002196C770E9CFDF91CF911F910895409136
:101620005002509151026091520270915302809188
:101630005402909155020C940709EF92FF920F9378
:101640001F93CF93DF938091550282958F7009F09D
:1016500065C080915202882309F460C080911E0207
:10166000F0901F02109150020091510260915302BC
:101670007091540291E01F3F09F090E0C091000189
:10168000D0910101292F96E0E92E8F1509F446C06B
:101690006115710521F00F3F21F030E003C031E00A
:1016A00001C0322F90E030FD36C0E89EF001E99E87
:1016B000F00D1124DF01A05EBD4F11963C911197F2
:1016C000301329C03C91311326C012963C911297D9
:1016D000311121C013964D915C911497461B570B05
:1016E0004C175D07C0F4809155028F708061809324
:1016F0005502EB5DFD4F80818F708061808380E5B6
:1017000092E00E948508DF91CF911F910F91FF9089
:10171000EF900C94EE0A01968770B7CFDF91CF91CE
:101720001F910F91FF90EF9008959F92AF92BF92FB
:10173000CF92DF92EF92FF920F931F93CF93DF939D
:10174000CDB7DEB761970FB6F894DEBF0FBECDBF41
:101750008C0185E0F801DE011D9601900D928A95BD
:10176000E1F7D8011296EC9090915002E09151026D
:1017700020915302309154022115310531F0EF3F91
:1017800031F481E09F3F19F403C081E001C080E0A3
:10179000B82FB1709B2E80FD47C1D8014C91119696
:1017A0005C9111971396AD90BC90149780E5C82E6C
:1017B00082E0D82EF0905202B501621B730B20918B
:1017C000000130910101FF2009F4D9C08091550238
:1017D0006217730708F095C0282F207F09F052C0C8
:1017E0005E1313C0491311C0FE2CE1100EC08F70A0
:1017F0008061809355020E940F0BC6010E948508EC
:1018000080915502F80185834DC1AB2831F05F3FCF
:1018100031F481E04F3F19F403C081E001C080E062
:1018200080FD03C081E08E2502C080E090E0F82FAB
:10183000F170FF2E80FF1CC080911E0220911F02BC
:1018400036E0821709F40BC190E0389FF001399F10
:10185000F00D1124E05EFD4F6181561306C06081DA
:10186000461303C06281E61203C001968770E9CF78
:10187000FE2CEE2009F416C1809155028160809300
:10188000550254C05E1306C0491304C0E11002C0E3
:10189000F80199C0C8010E94F008882361F1EE2088
:1018A00051F120915502822F82958F7090E002971E
:1018B00074F0809150029091510298878F8319861D
:1018C000BB86AA862C87CE0107960E94850886E0F3
:1018D000F801A0E5B2E001900D928A95E1F70E942F
:1018E0001D0B0E940F0B0AC05E1711F1C8010E9468
:1018F000F00881112CC0C8010E948508FF24F394D0
:10190000D1C0282F207F81F77A2DB98AA88A6E2D21
:1019100089890E94F80880E592E00E94850886E0A7
:10192000D6011D928A95E9F70E940F0BF12CBAC0DF
:101930004913DCCFE110DACFF8018583C8010E949A
:10194000850886E0D6011D928A95E9F7ABC0EE20A6
:1019500091F220915502822F82958F7090E002972C
:101960000CF4B5CF80915002909151029A838983F3
:101970001B82BD82AC822E83CE010196A6CF621758
:10198000730708F044C0FE2CEE2009F4B4CF5E13B8
:1019900030C049132EC02091550220FD21C0822F56
:1019A00082958F70482F50E041155105C9F0F8011C
:1019B00025834F30510541F08F5F982F9295907F8E
:1019C000822F8F70892B8583C8010E94850886E04D
:1019D000F801A0E5B2E001900D928A95E1F73CC0D4
:1019E00086E0F801A0E5B2E001900D928A95E1F75A
:1019F00059C0C8010E94F008811169CF8091550239
:101A0000816080935502C8010E9485084BC07A2DE1
:101A1000B98AA88A6E2D89890E94F80886E0D601C5
:101A20001D928A95E9F718C0EE2009F464CFC80129
:101A30000E94F008F82E882309F45DCF86E0F801B3
:101A4000A0E5B2E001900D928A95E1F780E592E081
:101A50000E947E050E941D0B0E940F0B23C04D8724
:101A60005E878D859E850E94C00A292F22952F7042
:101A7000223028F49F7039F0811105C00BC024304A
:101A800028F49F7049F4805E883020F0C8010E94DD
:101A900085089F2CF92C06C0D80115969C91907F43
:101AA00091F7F8CF8F2D61960FB6F894DEBF0FBE79
:101AB000CDBFDF91CF911F910F91FF90EF90DF90FD
:101AC000CF90BF90AF909F9008951F93CF93DF93D7
:101AD000CDB7DEB72C970FB6F894DEBF0FBECDBFE3
:101AE0004F83588769877A878B879C87CE010796B3
:101AF0000E94950B8823D1F09F8188852A853B859C
:101B0000232B31F08F3F31F481E09F3F19F403C064
:101B100081E001C080E080FD47C04F815885698524
:101B20007A858B859C850E9407093EC086E0FE0170
:101B30003796DE01119601900D928A95E1F7FF81AB
:101B4000E8856A857B856115710531F0EF3F31F4D9
:101B500081E0FF3F19F403C081E001C080E080FD17
:101B600023C020911F0230E0C90101968770992798
:101B700040911E0250E084179507F1F1F983EA8342
:101B80007D836C8396E0929FD001939FB00D1124CA
:101B9000A05EBD4FFE01319601900D929A95E1F73E
:101BA00080931F020E94EE0A16E080911E0290911F
:101BB0001F02891771F1189FC0011124805E9D4F8B
:101BC0000E94950B882329F1E0911E021E9FF001CF
:101BD0001124E05EFD4F40815181628173818481D7
:101BE00095810E94070980911E0290E001968770FE
:101BF000992780931E02D9CF0E94D10810921F020C
:101C000010921E02E0E5F2E086E0DF011D928A9567
:101C1000E9F72C960FB6F894DEBF0FBECDBFDF916B
:101C2000CF911F91089580915E0285958595859548
:101C3000089580915E028770089590915E0297707A
:101C400081E009F480E008958091690208959091FF
:101C50006902892B809369020895809590916902A9
:101C600089238093690208951092690208959091E2
:101C70006802892B8093680208958095909168028C
:101C800089238093680208951092680208958091D4
:101C90005F02089508950C944A0E0C944B0E909197
:101CA000EB0292FD08C090915F02981721F080939B
:101CB0005F020C944D0E089580915F02882329F0F5
:101CC00010925F0280E00C944D0E0895CF93DF9345
:101CD000E0910201F0910301809169028083E0911B
:101CE0000201F0910301908180916802892B808329
:101CF00080915F02882381F0E0910201F09103015D
:101D00009081892B808380910201909103010E9430
:101D1000C41F81110E945C0EC0910201D091030189
:101D200048E050E066E572E0CE010E94FC28892B75
:101D300069F088E0FE01A6E5B2E001900D928A9577
:101D4000E1F7CE01DF91CF910C94411FDF91CF914C
:101D500008950C944A0E9091EB0292FD10C098E009
:101D6000899F90011124262B20935E020E948909ED
:101D700080915E028595859585950C94A90E0C94AD
:101D8000890910925E0280E00C94A90E20915E02F7
:101D90008095822380935E02982F977099F430E0AB
:101DA000482F082E000C550B2417350759F0909139
:101DB000EB0292FD07C08595859585950E94AA093D
:101DC0000C94C10E0895CF939091EB0292FB2227C1
:101DD00020F92817F9F0C82F892FC0FB82F98093CA
:101DE000EB028091EA029091EB020E94450F82E0A3
:101DF0000E94C60E80918A0280FF0CC01F92CF9372
:101E000085E993E09F938F930E94DD030F900F90DD
:101E10000F900F90CF9108958091EB0282FB88275D
:101E200080F991E089270C94E30E81E00C94E30E95
:101E300080E00C94E30E6FEF7FEF80E090E00C9475
:101E40003E2980E090E00E941A2921E0893E9E4FC1
:101E500009F020E0822F089582E090E00C9412298E
:101E600083E090E00C941229CF9384E090E00E94EC
:101E70001229C82F82E290E00E9412292C2F30E014
:101E8000A901582BCA01CF910895CF93C92F682F6C
:101E900084E090E00E9420296C2F82E290E0CF91B4
:101EA0000C942029AB01BC018FE090E00C94322906
:101EB000AB01BC0183E190E00C94322960E070E05A
:101EC000CB010C94580F60E070E0CB010E94520FE0
:101ED0000C945E0F69EE7EEF80E090E00E943E2958
:101EE00060E082E090E00E94202960E083E090E0E2
:101EF0000E94202910921A0210921B0210921C02BA
:101F000010921D0260E084E090E00E94202960E0D1
:101F100082E290E00E94202960E085E090E00E944B
:101F2000202960E086E090E00E9420296FEF87E0A2
:101F300090E00E94202940E050E0BA0188E090E063
:101F40000E94322960E08DE090E00E94202940E06C
:101F500050E0BA0188E190E00E94322960E087E118
:101F600090E00E94202940E050E0BA018CE190E02E
:101F70000E94322960E070E080E290E00E943E29F9
:101F800040E050E0BA0188E190E00E9432290C94D0
:101F9000630F0C946A0F682F8EE090E00C94202958
:101FA0000E94B92060938602709387028093880212
:101FB00090938902609382027093830280938402DB
:101FC00090938502089585B7806885BF85B780683E
:101FD00085BF08950C94891508950C94EC0F0C940A
:101FE000EC0F0C94EF0F0C94EC0F0C94F30F0C947B
:101FF000EC0F0E94E30F8AEF92E20E94241F0E94DE
:10200000F70F0C94F50F0E94ED0F0C94EC0F0E944B
:102010002B130C94F1040E94A4200E94BF120E9472
:10202000A1150E94CD140E9407100E940A1B0E9455
:10203000AB150C94F10F5F926F927F928F929F92EB
:10204000AF92BF92CF92DF92EF92FF920F931F93C6
:10205000CF93DF93CDB7DEB72A970FB6F894DEBFE4
:102060000FBECDBF0E94F114C82E81110E94D00F67
:102070003AE6832E32E0932E00E010E0502E802FBF
:102080000E944F135C01F401619071904F0168262A
:10209000792661147104B1F40F5F1F4F0C301105E4
:1020A00069F78FEF89838A831B820E94AD2081604C
:1020B000782F9D838C8349815A816B818D810E9409
:1020C00034053AC080918A0281FD0E945813D12CB8
:1020D000EE24E394F12CC3018E219F21892B29F159
:1020E0000E94EA0F8823A9F0DE825F82AE20BF2023
:1020F00081E0AB2809F480E088870E94AD208160F0
:10210000782F9A8789874E815F8168858A850E94AA
:102110003405000F111FF801E659FD4F80819181B0
:10212000E826F926F182E08207C0D394EE0CFF1C6A
:10213000F9E0DF12D0CFB0CF81E0C11001C080E064
:102140002A960FB6F894DEBF0FBECDBFDF91CF91B8
:102150001F910F91FF90EF90DF90CF90BF90AF90C5
:102160009F908F907F906F905F9008950E941B10BA
:102170000E9489150E94E9190C940205CF93DF9300
:102180000E94E811EC01811521E5920708F045C095
:10219000811530E5930708F094C0883E910528F535
:1021A000803E910508F0F8C0883A910570F4853AB0
:1021B000910508F07CC08130910509F475C008F4E0
:1021C000E8C0049708F0E8C0E4C08F3B910508F030
:1021D000E0C0C85AD0E0CC0FDD1FCD59DE4F0990CA
:1021E000D881C02DCE019464D8C0811540E29407F7
:1021F00058F4811551E0950708F0CEC08D3E910549
:1022000008F4C7C09065C9C0C11580E4D80708F4B8
:10221000C0C0DF70CE01906AC0C0811525E592076D
:10222000A8F4811534E5930708F095C0811543E5BE
:10223000940708F07BC0811552E5950708F061C04E
:10224000D82FCC27CE01816F906AA7C0C11589E530
:10225000D807A0F4C11528E5D20708F082C0C1153F
:1022600036E5D30708F095C08C2F0E947C128F7141
:1022700090E0D82FCC27CE0190628FC0C1154AE5DF
:10228000D40708F474C0CE0190568115904208F02E
:1022900080C08D2F8F710E947C12DD27D0628F71DC
:1022A000AE01582BCA0179C081E090E076C0C55AD2
:1022B000D0E0CF56DE4F8881C82FD0E0CE019064A9
:1022C0006CC074E0969587957A95E1F7282F237076
:1022D0003C2F337081E090E002C0880F991F3A953F
:1022E000E2F79C68AC01522B9A019C2F9F70969547
:1022F000969550E2959FE0011124C9018C2B9D2BEE
:102300004CC08370992721E030E002C0220F331FB8
:102310008A95E2F79C2F9695969580E2989FE0012A
:102320001124C22BD32BCE019C6837C08370992710
:1023300021E030E002C0220F331F8A95E2F79C2F84
:102340009695969540E2949FE0011124C22BD32BE1
:10235000CE019A6822C0D82FCC27CE01846F906A14
:102360001CC0DC2FCC27CE01806F906A16C08C2F4A
:102370008F700E947C1294E0D695C7959A95E1F7EC
:10238000CF70D0E0DC2FCC27D0699E01282BC9016B
:1023900004C080E090E001C0CE01DF91CF910895AC
:1023A0002CE6829FC0011124FC0129E0729FE00D00
:1023B000F11D1124E60FF11DEE0FFF1FE852FF4F34
:1023C0008591949108950E94D0110E94BE100895A5
:1023D0008238910569F1B0F48133910509F46DC03B
:1023E00048F48932910509F463C08A32910509F4F1
:1023F00069C008958533910509F455C08933910565
:10240000B9F00895833E910569F138F4803E910555
:10241000B1F0823E910509F10895863E9105A9F13A
:10242000873E9105B9F1843E910509F064C023C04F
:102430002091EA0220FD4FC021FD4DC008958091FA
:10244000EA0280FD44C08091EB0280FF44C080918D
:10245000EA0284FD42C083EE4DC08091EA0282FF11
:1024600038C0F5CF8091EA0282FD33C08091EB0243
:1024700080FD31C0ECCF8091EB0281FF32C08091B2
:10248000EA0284FD2AC087EE35C08091EA0283FF0C
:1024900026C0F5CF8091EA0283FD21C08091EB0236
:1024A00081FD1FC0ECCF8091EA0285FD1CC01DC0DC
:1024B0008091EA0285FD19C016C08091EA0286FD6E
:1024C00016C017C08091EA0286FD13C010C089E3D0
:1024D00011C082EE0FC080EE0DC080E00BC086EE12
:1024E00009C084EE07C089E205C085E303C08AE223
:1024F00001C081E390E008959091EA0292FF0DC03F
:10250000282F2871283019F4877F846006C0282F6F
:102510002471243011F48B7F886093FF0DC0282F25
:102520002871283119F4877E846106C0282F247110
:10253000243111F48B7E88612091EB0220FF0DC0C5
:10254000382F3871383019F4877F816006C0382FF2
:102550003171313011F48E7F886021FF0DC0282F3A
:102560002871283119F4877E816106C0282F2171D6
:10257000213111F48E7E886194FD877E089510923A
:10258000E6021092E7021092E8021092E902089522
:10259000CF92DF92EF92FF926B017C010E9489152E
:1025A00081110EC00E94B920C61AD70AE80AF90A9A
:1025B000C092E602D092E702E092E802F092E902CD
:1025C000FF90EF90DF90CF9008950F931F930E949C
:1025D0008915882321F01F910F910C94B9200E9436
:1025E000B9200091E6021091E7022091E8023091B3
:1025F000E902600F711F821F931F1F910F910895B1
:102600000C941B0FCF930E94F1148FE39CE9019768
:10261000F1F700C000000E94F1140E9482158111A0
:1026200002C0C5E001C0C0E080E00E944F1321E07D
:1026300030E002C0220F331FCA95E2F782239323B2
:10264000892B29F00E940013CF910C941621CF9171
:1026500008950C9402130E94210F811102C00E9460
:10266000C90F0E942C0F80938A020E94340F90930E
:10267000EB028093EA020E9429130E94300F682F18
:1026800070E080E090E00E9429096091160270914C
:10269000170280911802909119020C946109E82F99
:1026A000F0E0EE0FFF1FEB5FFC4F808191810895FA
:1026B000CF92DF92EF92FF920F931F93CF93DF930E
:1026C0008AEB93E00E94440385E0E82E83E0F82E35
:1026D000C0E0D0E095EBC92E93E0D92E0CEA13E0D0
:1026E000DF93CF93DF92CF920E94DD0382EB93E0E2
:1026F0000E944403F701819191917F010E94D704C8
:102700009F938F931F930F930E94DD038AEA93E0B8
:102710000E94440321968DB79EB708960FB6F89491
:102720009EBF0FBE8DBFCC30D105D1F6DF91CF91CA
:102730001F910F91FF90EF90DF90CF90089580EA66
:102740008A95F1F7089500C008950C949F13089599
:102750000C94A7130C94A8130C94A7130C94AC130B
:102760000C94A713FF920F931F93CF93DF93CDB7D2
:10277000DEB72C970FB6F894DEBF0FBECDBF0E9418
:10278000891560911D03882309F443C05CE0F52E90
:102790008E010F5F1F4FF8018F2D11928A95E9F777
:1027A000862F90E0880F991FB8018B5F9C4F0E9485
:1027B000B915882399F08091EC0290E0880F991F59
:1027C0004CE050E0B8018B5F9C4F0E94FC2821E058
:1027D00020938B02892B61F410E018C080918B024A
:1027E0008823D1F3F8011192FA94E9F710928B0241
:1027F000A091EC02B0E0AA0FBB1FAB5FBC4F8CE016
:10280000F80101900D928A95E1F711E00E943A04D7
:1028100011C08091EC0270E0660F771F6B5F7C4FF8
:1028200090E0880F991F8B5F9C4F0E9455160E9465
:10283000B01310E0812F2C960FB6F894DEBF0FBEB8
:10284000CDBFDF91CF911F910F91FF900895F89424
:10285000E82FE295EF70F0E031A1282F2F7081E092
:1028600090E001C0880F2A95EAF7982F909593235E
:1028700091A392A1892B82A3789408950F931F931B
:10288000CF93DF93CDE9D1E089918F3F11F00E9482
:10289000271481E0C33AD807B9F7C4E9D1E00DE9BC
:1028A00011E089918F3F11F00E9427140C171D072A
:1028B000C1F7DF91CF911F910F910895BF92CF92F1
:1028C000DF92EF92FF920F931F93CF93DF938C01D0
:1028D000C62FD0E0CE0183569E4F6C01FC01908143
:1028E0009F3F09F450C0B62EF894E92FE295EF709F
:1028F000F0E081A19F7021E030E001C0220F9A95A5
:10290000EAF7822B81A382A12095282322A3789421
:102910000E94A313E4E9F1E04DE951E021E030E049
:10292000E12CF12C61916F3F89F0A62FA295AF7039
:10293000B0E090968C9190E06F7002C0959587956D
:102940006A95E2F780FD02C0C90102C080E090E014
:10295000E82AF92A220F331F4E175F0719F7F601ED
:1029600080818F3F11F00E94271461E0E114F1048F
:1029700009F460E08B2D0E94A513CC0FDD1FC00F62
:10298000D11FF982E882DF91CF911F910F91FF90C3
:10299000EF90DF90CF90BF900895809104018091D7
:1029A0000401811102C096E001C090E090931D03E4
:1029B00086E0891B8093EC020E943E1488E1E5E0EA
:1029C000F3E0DF01982F1D929A95E9F7EDEEF2E022
:1029D000DF011D928A95E9F786E00E9447150C9465
:1029E0003804EF92FF920F931F93CF93DF93CDB7ED
:1029F000DEB768970FB6F894DEBF0FBECDBF8E016D
:102A00000F5F1F4F88E1F80111928A95E9F7F12CC9
:102A10006F2DC8010E945E14F394F6E0FF12F8CF08
:102A200048E150E0B8018DEE92E00E94FC287C0164
:102A300021E0892B09F420E0E114F10441F088E160
:102A4000F801ADEEB2E001900D928A95E1F7609148
:102A50001D0370E0660F771F6B5F7C4F46E08DEEC5
:102A600092E00E944815EF2819F40E94B21302C0A8
:102A700081E090E068960FB6F894DEBF0FBECDBF40
:102A8000DF91CF911F910F91FF90EF9008950895DE
:102A9000FF920F931F93CF93DF93F82E092F162FDA
:102AA000D72FC42F222349F081E080938E020E9409
:102AB000AD2090938D0280938C0280918E028823AA
:102AC000D9F080918C0290918D020E94C5200597CB
:102AD00098F0EF2DF02FA12FBD2F80E090E04C2F2C
:102AE00050E08417950734F4219131912D933D9353
:102AF0000196F7CF10928E02DF91CF911F910F9127
:102B0000FF90089523982B9883B183FB882780F941
:102B100008958091910281110DC00E94B528811104
:102B200002C082E001C081E080939102823011F402
:102B30000E94B02881E090919102913009F080E0EC
:102B400008950E948215809304010E9489158111C5
:102B50000C94031608950E948915811102C00C94EB
:102B60000516089581E0909192029A3008F080E075
:102B70000895EF92FF920F931F93CF938C017B01E7
:102B8000C0919202CA3038F4B701C8010E945316AE
:102B9000811126C00AC080918F02909190020E94FC
:102BA000C520843F914080F719C0809192028F3FE9
:102BB00019F08F5F80939202809192028A30E0F048
:102BC0000E94AD209093900280938F0280918A02A0
:102BD00080FF04C084EE93E00E94440380E00DC0B7
:102BE000CA3040F080918A0280FF04C081ED93E0FA
:102BF0000E9444031092920281E0CF911F910F91A5
:102C0000FF90EF9008950C94BD1D0C94C01DDF92B1
:102C1000EF92FF920F931F93CF93DF937901C82F09
:102C2000880FDD0B41155105A9F0FE0193E0EE0F71
:102C3000FF1F9A95E1F7EB5FFE4F818192818D56E0
:102C40009D4F208130E04217530708F49A01A901F3
:102C50000E940929CE010E94A91ED82E8823D1F0F6
:102C600001151105B9F083E0CC0FDD1F8A95E1F75E
:102C7000FE01EB5FFE4F438150E00417150708F497
:102C8000A801CB5FDE4F6C817D816D567D4FC70102
:102C90000E9409298D2DDF91CF911F910F91FF90F7
:102CA000EF90DF9008950C948C170C94AC170F9351
:102CB0001F93CF93DF9300D000D0CDB7DEB76091E4
:102CC000B8027091B9028091BA029091BB020E9441
:102CD000D420643671058105910528F10E94E51222
:102CE000DC01CB010296A11DB11D89839A83AB83C0
:102CF000BC8300E010E020E030E044E050E0BE01A2
:102D00006F5F7F4F82E00E940716182F882361F0C3
:102D10000E94B9206093B8027093B9028093BA02FE
:102D20009093BB0201C011E0812F0F900F900F9084
:102D30000F90DF91CF911F910F9108958F929F92E5
:102D4000AF92BF92CF92DF92EF92FF920F931F93B9
:102D5000CF93DF937C015B01942E852E69010E9445
:102D6000B215811103C001E010E002C00AE010E0DA
:102D7000C1E0D0E0F894B501C701F6010995789457
:102D8000811129C021960C171D078CF0CC9F900152
:102D9000CD9F300D300D112480E090E045E34A9541
:102DA000F1F70000019628173907C1F7E3CF90919A
:102DB0008A02892F817090FF0FC08F929F928AE1C3
:102DC00094E09F938F930E94DD030F900F900F90DC
:102DD0000F9080E001C081E0DF91CF911F910F91B2
:102DE000FF90EF90DF90CF90BF90AF909F908F902B
:102DF0000895AF92BF92CF92DF92EF92FF920F931E
:102E00001F93CF93DF93CDB7DEB72D970FB6F8940E
:102E1000DEBF0FBECDBF7B01C090A301D090A40147
:102E200001E010E09E01235F3F4F40E050E060E092
:102E300070E080E00E940716182F882309F43EC036
:102E400056018FEFA81AB80A6091B4027091B502CA
:102E50008091B6029091B7020E94D4206436710529
:102E60008105910518F10CE010E09E012F5F3F4FA6
:102E700040E050E060E070E081E00E940716182F0B
:102E80006CE070E0C5010E940B1B91E02D852813BA
:102E900090E0192339F10E94B9206093B402709335
:102EA000B5028093B6029093B70211C06CE070E057
:102EB000C5010E940B1B9D858913D5CF8CE0F601BF
:102EC0003196DE01119601900D928A95E1F711235A
:102ED00049F08CE0FE013196A8EAB2E001900D9233
:102EE0008A95E1F78CE0E8EAF2E0D70101900D92D3
:102EF0008A95E1F7812F2D960FB6F894DEBF0FBEAD
:102F0000CDBFDF91CF911F910F91FF90EF90DF9098
:102F1000CF90BF90AF9008950F931F93CF93DF93FF
:102F2000EC018B0129EF36E145EA51E00E949E1643
:102F3000882361F027E536E142EB51E0B801CE018C
:102F4000DF91CF911F910F910C949E1680E0DF913D
:102F5000CF911F910F9108950F931F93CF93DF93FC
:102F6000F894C091A301D091A401CE0101962CE068
:102F7000FB01DC0101900D922A95E1F76CE070E015
:102F80000E940B1B88837894F8946D857E858F85CD
:102F900098890091A4021091A5022091A602309177
:102FA000A702601771078207930751F06093A4028C
:102FB0007093A5028093A6029093A7020E94C81264
:102FC0007894DF91CF911F910F9108950E947623FD
:102FD0000E940B100C9482230E9486230E94B6103C
:102FE0000C94A4230E944B200E945D230E94F90FA1
:102FF0000E94E6170E94EC170E940310FBCF8091FD
:10300000C20280FF06C06091220170E0660F771F48
:1030100026C081FF04C06091220184E005C082FFC8
:1030200007C06091220188E0689FB001112417C099
:103030009091C1029923D1F060912101961788F7F0
:103040002091220188E0289F90011124929FA001E5
:10305000939F500D112470E0CA010E94CE28603861
:10306000710540F46115710519F406C068E070E05F
:10307000862F08958FE7089581E008958091C20218
:1030800080FF08C060911E0170E075956795759589
:10309000679521C081FF06C060911E0170E07595A3
:1030A000679519C082FF04C060911E0170E010C0D6
:1030B0009091C002992399F060911D019617A0F795
:1030C00080911E01899FC001112470E00E94CE28CA
:1030D0006038710540F46115710519F406C061E0AE
:1030E00070E0862F08958FE7089581E008958D3E62
:1030F00021F40E94FF17819504C08E3E29F40E949E
:10310000FF178093C60208958F3E21F40E94FF1797
:10311000819504C0803F29F40E94FF178093C50267
:103120000895893F19F40E943E1805C08A3F31F482
:103130000E943E1881958093C70208958B3F21F429
:103140000E943E18819504C08C3F29F40E943E18CD
:103150008093C80208959FE0980F983078F421E09A
:1031600030E0A90102C0440F551F9A95E2F7CA0149
:103170009091C402892B8093C40208958D3F21F45D
:103180008091C20281600BC08E3F21F48091C20207
:10319000826005C08F3F29F48091C20284608093D1
:1031A000C20208958D3E39F49091C60297FF35C052
:1031B0001092C60259C08E3E29F49091C60219168B
:1031C000BCF32BC09091C5028F3E29F497FF25C018
:1031D0001092C50249C0803F19F41916CCF31DC0E6
:1031E0009091C702893F29F41916BCF41092C702C6
:1031F0003BC08A3F19F497FF10C0F8CF8B3F39F4DA
:103200009091C80297FF09C01092C8022DC08C3F50
:1032100021F49091C8021916BCF39FE0980F9830E2
:1032200080F421E030E0A90102C0440F551F9A95B7
:10323000E2F7CA0180959091C40289238093C40269
:1032400013C08D3F21F48091C2028E7F0BC08E3F50
:1032500021F48091C2028D7F05C08F3F29F48091B7
:10326000C2028B7F8093C2028091C502811106C089
:103270008091C602811102C01092C1028091C702E2
:10328000811106C08091C802811102C01092C00253
:10329000089580918A0283FF7EC087E594E00E94B2
:1032A00044038091C4021F928F9382E594E09F9320
:1032B0008F930E94DD0380E594E00E944403809197
:1032C000C502282F082E000C330B3F938F938DE4FB
:1032D00094E09F938F930E94DD038BE494E00E941F
:1032E00044038091C602282F082E000C330B3F9315
:1032F0008F9388E494E09F938F930E94DD0386E48C
:1033000094E00E9444038091C702282F082E000CED
:10331000330B3F938F9383E494E09F938F930E94AA
:10332000DD0381E494E00E9444038091C802282FC9
:10333000082E000C330B3F938F938EE394E09F9302
:103340008F930E94DD038BE394E00E9444038091FD
:10335000C1021F928F9388E394E09F938F930E9402
:10336000DD0386E394E00E9444038091C2021F9231
:103370008F9383E394E09F938F930E94DD0380E318
:1033800094E00E9444038DB79EB74C960FB6F89414
:103390009EBF0FBE8DBF0E94AD202091C50221119E
:1033A00004C02091C602222321F09093BF02809393
:1033B000BE022091C702211104C02091C80222231D
:1033C00021F09093BD028093BC0283EC92E00C94B8
:1033D0008A1FEF92FF920F931F93CF93DF9300D03A
:1033E00000D000D0CDB7DEB786E0E3ECF2E0DE013E
:1033F000119601900D928A95E1F7E090C502F09048
:10340000C6020091C7021091C8021092C502109224
:10341000C6021092C7021092C802E11003C0FF203A
:1034200009F45DC08091BE029091BF020E94C52048
:10343000AC019091C102992339F02091230130E031
:103440002417350758F04BC0209124018AE0289FAB
:10345000900111242417350718F041C09F3F19F03F
:103460009F5F9093C102EE2061F00E94FF171E142F
:1034700014F09FEF01C091E0989F902D112490933C
:10348000C502FF2061F00E94FF171F1414F09FEF88
:1034900001C091E0989F902D11249093C602309125
:1034A000C5023323E1F02091C6022223C1F045EB8F
:1034B0003403C0011124992319F09093C50203C06D
:1034C00081E08093C50235EB2303C00111249923C9
:1034D00019F09093C60203C081E08093C6020111E7
:1034E00003C0112309F45DC08091BC029091BD021C
:1034F0000E94C520AC019091C002992339F020911F
:103500001F0130E02417350758F04BC020912001EF
:103510008AE0289F900111242417350718F041C034
:103520009F3F19F09F5F9093C002002361F00E94BB
:103530003E18101614F09FEF01C091E0989F902D57
:1035400011249093C702112361F00E943E181116B6
:1035500014F09FEF01C091E0989F902D112490935B
:10356000C8023091C7023323E1F02091C802222320
:10357000C1F045EB3403C0011124992319F0909355
:10358000C70203C081E08093C70235EB2303C0016B
:103590001124992319F09093C80203C081E080930D
:1035A000C8028091C50281110BC08091C6028111B1
:1035B00007C08091C702811103C08091C8028111A8
:1035C0000E944919EB82FC820D831E8386E0FE0176
:1035D0003196A3ECB2E001900D928A95E1F7269620
:1035E0000FB6F894DEBF0FBECDBFDF91CF911F9114
:1035F0000F91FF90EF900895E3ECF2E086E0DF0199
:103600001D928A95E9F71092C1021092C0021092A1
:10361000C20208950895FC01680F791F8FEF91E3AE
:10362000E617F70771F02191822728E030E087FF45
:1036300003C0880F892701C0880F21503109B9F7CD
:10364000EFCF0895CF93DF93EC01FB0182818823B4
:1036500009F43CC1C430FDE5DF0760F4CB3F9CE5D5
:10366000D90788F49E0122503C452431310508F0E9
:103670002EC109C0C236EDE5DE0729F0C63AFDE5E8
:10368000DF0709F024C10E94340F9093EB0280936E
:10369000EA02C1318CE5D80709F4C6C008F042C07F
:1036A000C930ECE5DE0709F49BC000F5C5308CE5B8
:1036B000D80709F485C078F4C330ECE5DE0709F4D7
:1036C00078C008F07AC0C230DC4509F0F5C08091BE
:1036D000EA028160EFC0C7309CE5D90709F478C0E1
:1036E00008F07AC08091EA028061E4C0CD30FCE548
:1036F000DF0709F487C058F4CB309CE5D90709F4FB
:1037000079C008F07BC08091EA0288606FC0CF303A
:10371000FCE5DF0709F480C008F082C08091EA026E
:10372000877FC8C0CE3F9CE5D90709F471C000F57A
:10373000C531FCE5DF0709F485C068F4C3319CE5B9
:10374000D90709F475C008F095C00E94D10880918E
:10375000EA028F77AFC0CC3FFCE5DF07A9F108F0A4
:1037600054C0CB3FDC4509F0A7C08091EB0240C0BC
:10377000C230EDE5DE0709F489C058F4C1158DE5C6
:10378000D80709F45AC008F069C08091EB02826042
:103790002FC0C236EDE5DE0709F47CC0C63AFDE570
:1037A000DF0709F481C0C330DD4509F085C080E042
:1037B0006EC08091EA0282607DC08091EA0216C0EC
:1037C0008091EA02886076C08091EB0282604FC0EF
:1037D0008091EA0280626EC08091EA0280646AC0D1
:1037E0000E94D1088091EA02806864C0846062C04F
:1037F00081603DC08091EA028E7F5CC08091EA02C8
:103800008D7F58C08091EA0216C08091EB0218C0EB
:103810008091EB028D7F2BC08091EA028F7E4AC09F
:103820008091EA028F7D46C08091EA028F7B42C080
:103830008091EA02877F8B7F3DC08091EB028D7F74
:103840008E7F15C08091EA0282FB222720F991E049
:10385000922790FB82F990FB83F92CC08091EB02B8
:10386000982F909591708E7F892B90FB81F9809392
:10387000EB0222C00E94D1088091EA0287FB222736
:1038800020F991E0922790FB87F914C081E00E9413
:10389000CB0F12C08091EA0284FB222720F991E02D
:1038A000922790FB84F906C08091EA02982F9095A8
:1038B00090FB80F98093EA028091EA029091EB02FA
:1038C0000E94450F0E94D10880E001C081E0DF9195
:1038D000CF910895CF93DF9386319C4541F5EB015D
:1038E0000E94240E982F8A812091020130910301B9
:1038F000882379F09A7A81E009F480E08093C90204
:10390000911102C069E201C065E3C9010E9406206D
:103910000AC08091C902811102C069E201C065E359
:10392000C9010E9408200E94660E80E001C081E06B
:10393000DF91CF9108950F931F93CF93DF93C42FFF
:10394000D22FFC0182818823C9F04093CC020E94CF
:10395000AD209093CB028093CA0280E28C0F883016
:1039600008F057C0C77081E001C0880FCA95EAF718
:10397000DF91CF911F910F910C942E068091CC0274
:10398000481330C08091CA029091CB020E94C5209A
:10399000883C910538F510E21D0FCD17B9F080E293
:1039A0008C0F883040F4C77081E001C0880FCA9541
:1039B000EAF70E943506183028F581E09D2F9770B0
:1039C00001C0880F9A95EAF70E942E06802F0E9468
:1039D00025061830F0F4D77081E001C0880FDA9521
:1039E000EAF70AC080E28C0F883098F4C77081E053
:1039F00001C0880FCA95EAF7DF91CF911F910F910F
:103A00000C943506802FDF91CF911F910F910C946C
:103A10002506DF91CF911F910F9108950F939C017F
:103A2000CB01243F4CE5340731F188F4293DFCE516
:103A30003F07D9F02A3D4CE5340779F1283D3C4554
:103A4000A9F506E221EE41EE68ED7CE52BC0263FAC
:103A5000FCE53F07E1F0A8F0273F3C4539F507E2D8
:103A600025EE46EE67EF7CE51DC007E225EE45EE4C
:103A700069ED7CE517C006E221EE40EE64EF7CE5DF
:103A800011C007E225EE44EE65EF7CE50BC006E2CF
:103A900021EE42EE66EF7CE505C008E221E045EE4E
:103AA0006AED7CE50E949B1C80E008C0FC018281DD
:103AB000882319F01092CC0201C081E00F91089583
:103AC0008EE14A9B02C08150E1F74A9BFECF0895E8
:103AD0005A9880E28A95F1F75A9A0895FC012AE0F3
:103AE0002A95F1F728E090E080E031E040E14A9546
:103AF000F1F7880F4A9B02C08160932700C0000045
:103B000040E14A95F1F7215089F720E12A95F1F734
:103B100029B100C0000030E13A95F1F722FB2227DD
:103B200020F992272081920F90830895EF92FF92BF
:103B30000F931F93CF93DF931F92CDB7DEB71982F8
:103B40008C017C01E60EF11C0E151F0551F00E9440
:103B5000601DCE0101960E946E1DF80181938F01B8
:103B6000F3CF81E09981911180E00F90DF91CF91A7
:103B70001F910F91FF90EF900895529A5A9A0895CD
:103B800052985A9AEA9AE9E6F0E080818F7C808325
:103B90000895615091E001C0990F6A95EAF720E01D
:103BA00031E0992361F0492F482319F05A9A2327CD
:103BB00001C05A9840E24A95F1F79695F2CF222338
:103BC00011F05A9A01C05A9880E28A95F1F75A98F2
:103BD0000895FF920F931F93CF93DF93EC018C0115
:103BE000060F111DC017D10741F0F9900E94681D02
:103BF00068E08F2D0E94C91DF5CFDF91CF911F91F5
:103C00000F91FF9008951F920F920FB60F921124FB
:103C10000F931F932F933F934F935F936F937F93D4
:103C20008F939F93AF93BF93EF93FF93CF93DF93C4
:103C30001F92CDB7DEB719820E94601DCE0101969A
:103C40000E946E1D082F069506950695902F969555
:103C50009570202F2570920F292F23709695969599
:103C6000920F877089135FC0898181115CC0043015
:103C700008F059C080E18A95F1F75A9A529A82E089
:103C80008A95F1F700C05A9888E0089F80011124B6
:103C9000D801AB5FBE4F1696ED91FC911797309708
:103CA000A9F06091A3017091A40114962D913C910B
:103CB0001597260F371F11968D919C911297680FBB
:103CC000791F13964C9113978C910995F801EB5F2E
:103CD000FE4F6381662351F08091A3019091A4016E
:103CE00024813581820F931F0E94E91D0E94681D67
:103CF00080E18A95F1F75A9852985A9A80E18A950C
:103D0000F1F7F801EB5FFE4F6081662351F080917F
:103D1000A3019091A40121813281820F931F0E94FF
:103D2000961D0E94601D0F90DF91CF91FF91EF9142
:103D3000BF91AF919F918F917F916F915F914F91C3
:103D40003F912F911F910F910F900FBE0F901F90D9
:103D500018950F931F93CF93DF93843091050CF048
:103D60006DC0EC01F894529A5A9885E08A95F1F763
:103D700000009C2F969595702C2F2570920F892FFF
:103D800083709695969523E0CC0FDD1F2A95E1F779
:103D9000980F8E01092B0E94681D84E08A95F1F727
:103DA00000C068E0802F0E94C91D80E18A95F1F76C
:103DB00052985A9A4A9902C000C0FCCF87E090E01E
:103DC0004A9B08C0019721F4529A5A9A789436C0B7
:103DD00000C0F6CFFE01EB5FFE4F6381662381F0EA
:103DE0008091A3019091A40124813581820F931FBA
:103DF0000E94961D811104C0529A5A9A78941FC04D
:103E00000E94601D80E28A95F1F75A98529A80E1EB
:103E10008A95F1F7CB5FDE4F6881662351F0809180
:103E2000A3019091A40129813A81820F931F0E94DE
:103E3000E91D0E94681D789481E001C080E0DF9157
:103E4000CF911F910F9108959093CD018093CC0154
:103E500008959093D3028093D20208950E94891509
:103E6000811103C08091CD020895E091D202F091BA
:103E7000D302309721F00190F081E02D099480E089
:103E80000895EF92FF920F931F93CF93DF93E091EA
:103E9000D202F091D3023097B1F18C010280F3810C
:103EA000E02D099580918A0282FF2DC080FF04C019
:103EB00082E894E00E944403E80118E08CE7E82ED1
:103EC00084E0F82E80918A0280FF0BC088811F92C7
:103ED0008F93FF92EF920E94DD030F900F900F904F
:103EE0000F90115021961111EDCF80918A0280FF21
:103EF0000AC08AE794E0DF91CF911F910F91FF9064
:103F0000EF900C944403DF91CF911F910F91FF909C
:103F1000EF900895E091D202F091D302309739F0FA
:103F200022E0DC012C930480F581E02D09940895B2
:103F30002091D0023091D1022817390771F0909367
:103F4000D1028093D002E091D202F091D302309757
:103F500021F00680F781E02D099408952091CE028A
:103F60003091CF022817390771F09093CF028093D8
:103F7000CE02E091D202F091D302309721F000847A
:103F8000F185E02D09940895FC01329697E080E0D8
:103F9000915029F021912223D9F38F5FF9CF089511
:103FA000662349F0FC01329608962191621729F0A8
:103FB000E817F907D1F780E0089581E008959C01A2
:103FC000FC0132969FEF80E04191461789F09F3FB8
:103FD00019F4411101C0982F8F5F8630A9F79F3FD8
:103FE00039F0F901E90FF11D97FDFA956283089503
:103FF00008959C012A5F3F4FFC014281461301C096
:104000001282019682179307B9F708950C94DF1F67
:104010000C94F91F029626E0FC0111922A95E9F70B
:10402000089508950C94112083E08093D4020C9499
:104030001220811102C081E001C082E08093D4028D
:104040000C9412200C94192081E08093D4020C94DB
:1040500012200C94242008950C942B200C942C20D6
:104060000C942B200C942B200C942B20CF930E948B
:1040700032200E94F1140E943020C0E08C2F0E9458
:104080004F13892B29F4CF5FCC30C1F780E001C0FA
:1040900081E0CF91089508951F920F920FB60F926D
:1040A00011248F939F93AF93BF938091D502811179
:1040B00013C080911E0390911F03A0912003B09123
:1040C00021034196A11DB11D80931E0390931F03F0
:1040D000A0932003B0932103BF91AF919F918F9143
:1040E0000F900FBE0F901F9018958091260384307B
:1040F00031F10E94BD041092D50220E488E190E0E5
:104100000FB6F894A895809360000FBE20936000CE
:1041100083B7817F846083BF83B7816083BF7894D6
:10412000889583B78E7F83BF0FB6F894A89580914A
:104130006000886180936000109260000FBE089557
:104140000E94D1080C94C10482E084BD93E095BD27
:104150009AEF97BD80936E0008952FB7F8948091E1
:104160001E0390911F03A0912003B09121032FBF44
:1041700008952FB7F89460911E0370911F038091EA
:104180002003909121032FBF08959C014FB7F8940D
:1041900080911E0390911F03A0912003B0912103F1
:1041A0004FBF821B930B0895CF92DF92EF92FF9245
:1041B0002FB7F894C0901E03D0901F03E090200307
:1041C000F09021032FBFA7019601261B370B480B48
:1041D000590BCA01B901FF90EF90DF90CF9008957D
:1041E00078941F920F920FB60F9211248F939F9382
:1041F000AF93BF9380911E0390911F03A091200362
:10420000B09121030196A11DB11D80931E039093CF
:104210001F03A0932003B0932103BF91AF919F91FF
:104220008F910F900FBE0F901F90189587E797E71B
:1042300090930108809300089AE088E10FB6F89403
:10424000A895809360000FBE90936000FFCF80918F
:10425000E4020895089522E02093E9002FEF3091C1
:10426000E800215035FD06C035ED3A95F1F7000024
:104270002111F5CF2091E80025FF0BC040E050E070
:1042800066E070E00E9413248091E8008E778093AE
:10429000E8000895CF93DF9321E02093E9002FEF0A
:1042A0003091E800215035FD06C035ED3A95F1F723
:1042B00000002111F5CF2091E80025FF14C0EC018A
:1042C00040E050E068E070E00E9413248091E80034
:1042D0008E778093E80088E0FE01ACEDB2E00190BB
:1042E0000D928A95E1F7DF91CF9108958093D802DE
:1042F0007093DA026093D90280912603843001F52D
:1043000082E08093E9008FEF9091E800815095FD65
:1043100006C095ED9A95F1F700008111F5CF8091D7
:10432000E80085FF0DC040E050E063E070E088EDFC
:1043300092E00E9413248091E8008E778093E80039
:104340000895BC0184E00C947621BC0183E00C94B8
:10435000762188EA94E00E9444038091250381112C
:1043600009C00E94A4250E9401268091E200846079
:104370008093E200089584EA94E00E94440310923E
:104380002503089580EA94E00E9444030C942920B8
:104390008CE994E00E9444036091220381E0611162
:1043A00001C080E00C94142088E994E00E9444034A
:1043B0009091260381E0943009F080E0609122031F
:1043C0000C9419202091D7022F5F822F62E30E9464
:1043D000C228992319F02093D70208951092D7028A
:1043E0008091DB02882371F180912603843041F5AE
:1043F0008091E9008F702091EC00922F917020FD48
:1044000090E8892B93E09093E9009091EB0090FF66
:1044100014C09091EE0097FF10C09091E80095FFB6
:1044200003C01092F100F9CF9091E80090FF05C011
:104430009091E8009E779093E8008F708093E90058
:104440001092DB02089542E061EC81E00E941D259C
:1044500042E261EC82E00E941D2542E261EC83E0D1
:104460000E941D259091260381E0943009F080E0A0
:10447000609122030C94222080912803833009F458
:1044800061C030F4813071F0823009F49AC008952F
:104490008A3009F486C08B3009F46CC0893009F089
:1044A000A8C020C080912703813A09F0A2C0809162
:1044B000E800877F8093E80080912B0390912C0384
:1044C000892B21F468E08CED92E003C060E080E08D
:1044D00090E070E00E945E248091E8008B778093EA
:1044E000E800089580912703813209F082C080910D
:1044F0002B0390912C03029708F07BC08091E80079
:10450000877F8093E8008091E80082FD05C080915C
:1045100026038111F8CF6DC02091F3008091F20045
:1045200090E0922B029731F48091F100813011F0EC
:10453000863021F48091F1008093E4028091E800BC
:104540008B7753C080912703813A09F052C0809144
:104550002B0390912C03892B09F04BC08091E8002C
:10456000877F8093E8008091E80080FFFCCF8091F6
:10457000310136C0809127038132D9F580912B0318
:1045800090912C03892BA9F58091E800877F809377
:10459000E8000E94522580912903809331010C94F8
:1045A000D10880912703813221F58091E800877F2F
:1045B0008093E8000E94522580912A038093E502AF
:1045C000089580912703813AA1F48091E800877FC4
:1045D0008093E8008091E80080FFFCCF8091E502A5
:1045E0008093F1008091E8008E778093E8000C942E
:1045F000522508959FB7F8941092DB029FBF9091C7
:104600002603943009F057C09091E9009F703091D3
:10461000EC00232F217030FD20E8922B23E0209323
:10462000E9002091EB0020FF43C02091EE0027FF1E
:104630003FC02091D602222321F02091E80025FFDF
:1046400037C01092D60226E03091E80035FD15C043
:1046500030912603343061F53091EB0035FD28C0F0
:10466000215021F481E08093D60222C0EFE9FFE0DF
:104670003197F1F700C00000E7CF8093F1008091FF
:10468000E80085FD0AC08091E80080FFFCCF8091A2
:10469000E8008E778093E80006C08FB7F89421E099
:1046A0002093DB028FBF9F709093E90080E0089514
:1046B0009F709093E9008FEF089584B7877F84BF40
:1046C0000FB6F894A895809160008861809360008F
:1046D000109260000FBE90E080E80FB6F8948093CF
:1046E0006100909361000FBE0C9424200E94A425C9
:1046F0000E940126E2EEF0E080818460808378945D
:104700000C94952885E291E00C94291F8091260352
:104710008530C9F484E994E00E9444038091260323
:10472000853079F40E947520809124038823B1F3A9
:104730000E943620882391F30E94FD230E94D10815
:10474000EDCF0C94A020089508950C94A723292F51
:10475000332723303105C9F060F42130310581F071
:104760002230310509F041C08BE590E028EE34E0BD
:1047700040C021323105E1F02232310531F135C03E
:1047800082E190E023E435E034C09927813091053F
:1047900049F028F0029749F5ECEAF4E005C0E4EEB0
:1047A000F4E002C0E6ECF4E0849190E09F0121C0C7
:1047B00063307105D0F4660F771FFB01EA53FE4F9B
:1047C0002081318189E090E014C06330710568F484
:1047D000FB01EE0FFF1FE054FE4F20813181FB01F2
:1047E000E354FE4F808190E004C080E090E020E040
:1047F00030E0FA0131832083089580E189BD82E1B0
:1048000089BD09B400FEFDCF8091D8008F7D8093D3
:10481000D8008091E00082608093E0008091E00009
:1048200081FDFCCF0895CF92DF92EF92FF920F931C
:104830001F93CF93DF93EC018B017A010E947125C6
:10484000811133C0E114F10439F0F70180819181C5
:10485000081B190BC80FD91FC12CD12C011511052C
:1048600019F18091E80085FD16C08091E8008E77EF
:104870008093E800E114F10449F0F701808191810F
:10488000C80ED91ED182C08285E00FC00E9471255A
:10489000882321F30AC089918093F1000150110906
:1048A000FFEFCF1ADF0ADACF80E0DF91CF911F91BF
:1048B0000F91FF90EF90DF90CF90089520912D03FE
:1048C00030912E032617370748F06115710539F42A
:1048D0002091E8002E772093E80001C0B901FC0187
:1048E00020E06115710579F1809126038823F1F1AB
:1048F0008530F1F18091E80083FD3CC08091E800B3
:1049000082FD2EC08091E80080FFEBCF2091F30064
:104910008091F20090E0922B6115710551F0883082
:10492000910538F421912093F100615071090196AD
:10493000F3CF21E0089709F020E08091E8008E771E
:104940008093E800CECF2111CFCF0AC080912603FB
:10495000882361F0853061F08091E80083FD0AC012
:104960008091E80082FFF2CF80E0089582E0089510
:1049700083E0089581E0089520912D0330912E0366
:104980002617370748F06115710539F42091E800C2
:104990002E772093E80001C0B901FC0120E06115E9
:1049A000710591F180912603882309F440C0853078
:1049B00009F43FC08091E80083FD3DC08091E8008C
:1049C00082FD2FC08091E80080FFE9CF2091F300A5
:1049D0008091F20090E0922B6115710559F08830BA
:1049E000910540F424912093F100319661507109B2
:1049F0000196F2CF21E0089709F020E08091E800CD
:104A00008E778093E800CBCF2111CCCF0AC0809164
:104A10002603882361F0853061F08091E80083FDF2
:104A20000AC08091E80082FFF2CF80E0089582E022
:104A3000089583E0089581E00895982F973068F5F0
:104A40009093E900981739F07091EC002091ED00F7
:104A50005091F00003C0242F762F50E021FD02C0BA
:104A60009F5FECCF3091EB003E7F3093EB003091B5
:104A7000ED003D7F3093ED003091EB0031603093DD
:104A8000EB007093EC002093ED005093F000209128
:104A9000EE0027FDE5CF80E008958F708093E90058
:104AA00081E008958091270387FF11C08091E8007D
:104AB00082FD05C0809126038111F8CF11C080913D
:104AC000E8008B770BC080912603882349F0809102
:104AD000E80080FFF8CF8091E8008E778093E800AF
:104AE00008952091E4003091E50095E64091EC00B6
:104AF000842F817040FF23C08091E80080FD1DC09D
:104B000080912603882399F0853099F08091EB00FD
:104B100085FD11C04091E4005091E5002417350750
:104B200029F3915011F09A01E1CF84E0089582E0D9
:104B3000089583E0089581E0089580E0089540910C
:104B4000E80042FFDDCF08950E9412260E941A2637
:104B5000E0EEF0E0808181608083E8EDF0E080812C
:104B60008F77808319BCA7EDB0E08C918E7F8C93FA
:104B700080818F7E80831092250308950F931F9369
:104B8000CF93DF930E9412260E941A26C8EDD0E030
:104B900088818F77888388818068888388818F7DEA
:104BA000888319BC109226031092220310922403CA
:104BB0001092230300EE10E0F80180818B7F808348
:104BC00088818160888342E060E080E00E941D254A
:104BD000E1EEF0E080818E7F8083E2EEF0E0808184
:104BE00081608083808188608083F80180818E7FEE
:104BF0008083888180618883DF91CF911F910F919D
:104C00000895E8EDF0E080818F7E8083E7EDF0E0AD
:104C100080818160808384E082BF81E0809325036E
:104C20000C94BE25E8EDF0E080818E7F80831092A9
:104C3000E20008951092DA001092E10008951F92A8
:104C40000F920FB60F9211242F933F934F935F93C0
:104C50006F937F938F939F93AF93BF93EF93FF9344
:104C60008091E10082FF0BC08091E20082FF07C0CB
:104C70008091E1008B7F8093E1000E94E22180918E
:104C8000DA0080FF1FC08091D80080FF1BC0809198
:104C9000DA008E7F8093DA008091D90080FF0DC00A
:104CA00080E189BD82E189BD09B400FEFDCF81E0CC
:104CB000809326030E94A92105C019BC10922603E7
:104CC0000E94BB218091E10080FF19C08091E20029
:104CD00080FF15C08091E2008E7F8093E20080917A
:104CE000E20080618093E2008091D800806280932E
:104CF000D80019BC85E0809326030E94C8218091CA
:104D0000E10084FF30C08091E20084FF2CC080E18C
:104D100089BD82E189BD09B400FEFDCF8091D80034
:104D20008F7D8093D8008091E1008F7E8093E10099
:104D30008091E2008F7E8093E2008091E2008160AA
:104D40008093E20080912203882311F084E007C061
:104D50008091E30087FD02C081E001C083E0809381
:104D600026030E94D4218091E10083FF29C0809115
:104D7000E20083FF25C08091E100877F8093E100FE
:104D800082E080932603109222038091E1008E7FBF
:104D90008093E1008091E2008E7F8093E200809119
:104DA000E20080618093E20042E060E080E00E94E7
:104DB0001D258091F00088608093F0000E94C22140
:104DC000FF91EF91BF91AF919F918F917F916F91E3
:104DD0005F914F913F912F910F900FBE0F901F90B9
:104DE00018951F920F920FB60F9211242F933F9395
:104DF0004F935F936F937F938F939F93AF93BF93E3
:104E0000CF93DF93EF93FF93C091E900CF70809130
:104E1000EC00D82FD17080FDD0E81092E90080918D
:104E2000F000877F8093F00078940E9435271092DD
:104E3000E9008091F00088608093F000CD2BCF7066
:104E4000C093E900FF91EF91DF91CF91BF91AF91B6
:104E50009F918F917F916F915F914F913F912F9192
:104E60000F900FBE0F901F9018951F93CF93DF9355
:104E7000CDB7DEB7AA970FB6F894DEBF0FBECDBF91
:104E8000E7E2F3E08091F100819323E0EF32F20753
:104E9000C9F70E943C228091E80083FF2EC18091D7
:104EA000270390912803492F50E04A30510508F01C
:104EB00024C1FA01EE59FF4F0C94E228803821F00A
:104EC000823809F01AC108C080912303909124030D
:104ED000992389F082600FC080912B038F708730F7
:104EE00008F00BC18093E9008091EB0085FB8827D7
:104EF00080F91092E9009091E800977F9093E80084
:104F00008093F1001092F100D1C0282F2D7F09F07D
:104F1000F4C0882319F0823061F0EFC0809129033A
:104F2000813009F0EAC0933009F080E080932403D7
:104F30002EC08091290381112AC080912B038F708C
:104F40002FEF280F263008F0D8C08093E900209179
:104F5000EB0020FF1CC0933021F48091EB008062B5
:104F600014C09091EB0090619093EB0021E030E051
:104F7000A90102C0440F551F8A95E2F74093EA0049
:104F80001092EA008091EB0088608093EB00109211
:104F9000E9008091E800877F8093E8000E94522515
:104FA000ACC08111AAC0109129031F778091E30042
:104FB0008078812B8093E3008091E800877F809345
:104FC000E8000E9452258091E80080FFFCCF80918C
:104FD000E30080688093E300111102C082E001C009
:104FE00083E08093260389C08058823008F085C012
:104FF0008091290390912A038C3D53E0950779F520
:1050000083E08A838AE289834FB7F894DE0113969E
:1050100020E03EE051E2E32FF0E050935700E491AE
:1050200020FF03C0E295EF703F5FEF708E2F90E09E
:10503000EA3010F0C79601C0C0968D939D932F5F04
:10504000243149F74FBF8091E800877F8093E800C3
:105050006AE270E0CE0101960E945E2416C0609163
:105060002B0370912C03AE014F5F5F4F0E94A5236D
:10507000BC01892B09F441C09091E800977F90937F
:10508000E80089819A810E94BC248091E8008B7796
:105090008093E80032C0803881F58091E800877FF6
:1050A0008093E800809122038093F1008091E800D2
:1050B0008E7772CF811121C08091290390912A03AC
:1050C00099270297D4F48091E800877F8093E800C5
:1050D00080912903809322030E945225809122030C
:1050E000811106C08091E30087FD02C081E001C00C
:1050F00084E0809326030E9423228091E80083FFAE
:105100000AC08091E800877F8093E8008091EB00DF
:1051100080628093EB00AA960FB6F894DEBF0FBEB4
:10512000CDBFDF91CF911F910895CF93809126033A
:105130008823A1F0C091E900CF709091EC00892FF5
:10514000817090FD80E8C82B1092E9008091E80002
:1051500083FD0E943527CF70C093E900CF91089559
:105160000E94A425109226030895E8EDF0E08081C6
:10517000806180838AE18A95F1F700C08091D9002F
:1051800081700895991B79E004C0991F961708F063
:10519000961B881F7A95C9F78095089597FB072E6F
:1051A00016F4009407D077FD09D00E94E82807FC88
:1051B00005D03EF4909581959F4F08957095619527
:1051C0007F4F0895EE0FFF1F0590F491E02D099495
:1051D000AA1BBB1B51E107C0AA1FBB1FA617B7071D
:1051E00010F0A61BB70B881F991F5A95A9F7809539
:1051F0009095BC01CD010895FB01DC0104C08D91A7
:105200000190801921F441505040C8F7881B990B38
:105210000895FB01DC0102C001900D924150504005
:10522000D8F70895F999FECF92BD81BDF89A9927D4
:1052300080B50895A8E1B0E042E050E00C94462922
:10524000262FF999FECF92BD81BDF89A019700B43F
:10525000021639F01FBA20BD0FB6F894FA9AF99ADF
:105260000FBE08950396272F0E9421290E9420290E
:10527000252F0E942129242F0C9421290196272FC4
:105280000E9421290C942029DC01CB01FC01F99911
:10529000FECF06C0F2BDE1BDF89A319600B40D9282
:0C52A00041505040B8F70895F894FFCF3B
:1052AC00C8006002010000000100000000000000C6
:1052BC000C01000000040D00000000000028085044
:1052CC00011E0A140127214A212B21A521A1212AE3
:1052DC002101E200E900EA00B500B600B700CD00FC
:1052EC008301CC008A019201940121022302240241
:1052FC002502260227022A02B300B4006F007000B8
:10530C00818283E200E900EA00B500B600B700CD67
:10531C00008301CC008A0192019401210223022412
:10532C00022502260227022A02B300B4006F007085
:10533C0000818283329190946697C63435F4F5F6E9
:10534C00F731369302736C6176655F6D61747269C7
:10535C00780073796E635F74696D657200407B22AF
:0C536C00F20577055505FA0413052C0521
:00000001FF
